 getstacktr06

 Timestamp is 9e363381 (reproducible build file hash)

 Preferred load address is 0000000180000000

 Start         Length     Name                   Class
 0001:00000000 00001fa0H .text$mn                CODE
 0001:00001fa0 00000036H .text$mn$00             CODE
 0001:00001fd6 00000092H .text$x                 CODE
 0002:00000000 000001a8H .idata$5                DATA
 0002:000001a8 00000038H .00cfg                  DATA
 0002:000001e0 00000008H .CRT$XCA                DATA
 0002:000001e8 00000008H .CRT$XCZ                DATA
 0002:000001f0 00000008H .CRT$XIA                DATA
 0002:000001f8 00000008H .CRT$XIC                DATA
 0002:00000200 00000008H .CRT$XIZ                DATA
 0002:00000208 00000008H .CRT$XLA                DATA
 0002:00000210 00000008H .CRT$XLZ                DATA
 0002:00000218 00000008H .CRT$XPA                DATA
 0002:00000220 00000008H .CRT$XPZ                DATA
 0002:00000228 00000008H .CRT$XTA                DATA
 0002:00000230 00000010H .CRT$XTZ                DATA
 0002:00000238 00000000H .gehcont$y              DATA
 0002:00000238 00000000H .gfids$y                DATA
 0002:00000240 000011c0H .rdata                  DATA
 0002:00001400 00000000H .rdata$CastGuardVftablesA DATA
 0002:00001400 00000000H .rdata$CastGuardVftablesC DATA
 0002:00001400 00000028H .rdata$T                DATA
 0002:00001428 00000064H .rdata$voltmd           DATA
 0002:0000148c 0000031cH .rdata$zzzdbg           DATA
 0002:000017a8 00000008H .rtc$IAA                DATA
 0002:000017b0 00000008H .rtc$IZZ                DATA
 0002:000017b8 00000008H .rtc$TAA                DATA
 0002:000017c0 00000008H .rtc$TZZ                DATA
 0002:000017c8 00000004H .tls                    DATA
 0002:000017cc 00000004H .tls$                   DATA
 0002:000017d0 00000008H .tls$ZZZ                DATA
 0002:000017d8 00000228H .xdata                  DATA
 0002:00001a00 00000078H .edata                  DATA
 0002:00001a78 00000064H .idata$2                DATA
 0002:00001adc 00000014H .idata$3                DATA
 0002:00001af0 000001a8H .idata$4                DATA
 0002:00001c98 00000454H .idata$6                DATA
 0003:00000000 00000210H .data                   DATA
 0003:00000210 000007a8H .bss                    DATA
 0004:00000000 00000294H .pdata                  DATA

  Address         Publics by Value              Rva+Base               Lib:Object

 0000:00000000       __AbsoluteZero             0000000000000000     <absolute>
 0000:00000000       ___safe_se_handler_count   0000000000000000     <absolute>
 0000:00000000       ___safe_se_handler_table   0000000000000000     <absolute>
 0000:00000000       __arm64x_extra_rfe_table   0000000000000000     <absolute>
 0000:00000000       __arm64x_extra_rfe_table_size 0000000000000000     <absolute>
 0000:00000000       __arm64x_native_entrypoint 0000000000000000     <absolute>
 0000:00000000       __arm64x_redirection_metadata 0000000000000000     <absolute>
 0000:00000000       __arm64x_redirection_metadata_count 0000000000000000     <absolute>
 0000:00000000       __dynamic_value_reloc_table 0000000000000000     <absolute>
 0000:00000000       __enclave_config           0000000000000000     <absolute>
 0000:00000000       __guard_check_icall_a64n_fptr 0000000000000000     <absolute>
 0000:00000000       __guard_eh_cont_count      0000000000000000     <absolute>
 0000:00000000       __guard_eh_cont_table      0000000000000000     <absolute>
 0000:00000000       __guard_fids_count         0000000000000000     <absolute>
 0000:00000000       __guard_fids_table         0000000000000000     <absolute>
 0000:00000000       __guard_iat_count          0000000000000000     <absolute>
 0000:00000000       __guard_iat_table          0000000000000000     <absolute>
 0000:00000000       __guard_longjmp_count      0000000000000000     <absolute>
 0000:00000000       __guard_longjmp_table      0000000000000000     <absolute>
 0000:00000000       __hybrid_auxiliary_iat     0000000000000000     <absolute>
 0000:00000000       __hybrid_auxiliary_iat_copy 0000000000000000     <absolute>
 0000:00000000       __hybrid_code_map          0000000000000000     <absolute>
 0000:00000000       __hybrid_code_map_count    0000000000000000     <absolute>
 0000:00000000       __x64_code_ranges_to_entry_points 0000000000000000     <absolute>
 0000:00000000       __x64_code_ranges_to_entry_points_count 0000000000000000     <absolute>
 0000:00000100       __guard_flags              0000000000000100     <absolute>
 0000:00000000       __ImageBase                0000000180000000     <linker-defined>
 0001:00000000       ?SetEventNotificationMode@_jvmtiEnv@@QEAA?AW4jvmtiError@@W4jvmtiEventMode@@W4jvmtiEvent@@PEAV_jobject@@ZZ 0000000180001000 f i libgetstacktr06.obj
 0001:0000000c       ?TranslateError@@YAPEBDW4jvmtiError@@@Z 000000018000100c f   libgetstacktr06.obj
 0001:0000032c       ?compare_stack_trace@@YAHPEAU_jvmtiEnv@@PEAUJNIEnv_@@PEAV_jobject@@QEAUframe_info@@HH@Z 000000018000132c f   libgetstacktr06.obj
 0001:00000ac4       Agent_OnLoad               0000000180001ac4 f   libgetstacktr06.obj
 0001:00000c1c       Breakpoint                 0000000180001c1c f   libgetstacktr06.obj
 0001:00000d1c       Java_getstacktr06_getReady 0000000180001d1c f   libgetstacktr06.obj
 0001:00000dc4       SingleStep                 0000000180001dc4 f   libgetstacktr06.obj
 0001:00000ea8       __local_stdio_printf_options 0000000180001ea8 f i libgetstacktr06.obj
 0001:00000eb0       printf                     0000000180001eb0 f i libgetstacktr06.obj
 0001:00000ff8       _Init_thread_footer        0000000180001ff8 f   MSVCRT:thread_safe_statics.obj
 0001:00001058       _Init_thread_header        0000000180002058 f   MSVCRT:thread_safe_statics.obj
 0001:000010c0       _Init_thread_notify        00000001800020c0 f   MSVCRT:thread_safe_statics.obj
 0001:00001104       _Init_thread_wait          0000000180002104 f   MSVCRT:thread_safe_statics.obj
 0001:00001168       __GSHandlerCheck           0000000180002168 f   MSVCRT:gshandler.obj
 0001:00001188       __GSHandlerCheckCommon     0000000180002188 f   MSVCRT:gshandler.obj
 0001:00001200       __security_check_cookie    0000000180002200 f   MSVCRT:amdsecgs.obj
 0001:00001540       _DllMainCRTStartup         0000000180002540 f   MSVCRT:dll_dllmain.obj
 0001:00001580       __scrt_acquire_startup_lock 0000000180002580 f   MSVCRT:utility.obj
 0001:000015bc       __scrt_dllmain_after_initialize_c 00000001800025bc f   MSVCRT:utility.obj
 0001:000015f0       __scrt_dllmain_before_initialize_c 00000001800025f0 f   MSVCRT:utility.obj
 0001:00001608       __scrt_dllmain_crt_thread_attach 0000000180002608 f   MSVCRT:utility.obj
 0001:00001630       __scrt_dllmain_crt_thread_detach 0000000180002630 f   MSVCRT:utility.obj
 0001:00001648       __scrt_dllmain_exception_filter 0000000180002648 f   MSVCRT:utility.obj
 0001:000016a8       __scrt_dllmain_uninitialize_c 00000001800026a8 f   MSVCRT:utility.obj
 0001:000016d8       __scrt_dllmain_uninitialize_critical 00000001800026d8 f   MSVCRT:utility.obj
 0001:000016ec       __scrt_initialize_crt      00000001800026ec f   MSVCRT:utility.obj
 0001:00001738       __scrt_initialize_onexit_tables 0000000180002738 f   MSVCRT:utility.obj
 0001:000017c4       __scrt_is_nonwritable_in_current_image 00000001800027c4 f   MSVCRT:utility.obj
 0001:0000185c       __scrt_release_startup_lock 000000018000285c f   MSVCRT:utility.obj
 0001:00001880       __scrt_uninitialize_crt    0000000180002880 f   MSVCRT:utility.obj
 0001:000018ac       _onexit                    00000001800028ac f   MSVCRT:utility.obj
 0001:000018e8       atexit                     00000001800028e8 f   MSVCRT:utility.obj
 0001:00001900       __crt_debugger_hook        0000000180002900 f   MSVCRT:utility_desktop.obj
 0001:00001908       __scrt_fastfail            0000000180002908 f   MSVCRT:utility_desktop.obj
 0001:00001a54       _guard_check_icall_nop     0000000180002a54 f i MSVCRT:guard_support.obj
 0001:00001a58       __raise_securityfailure    0000000180002a58 f   MSVCRT:gs_report.obj
 0001:00001a8c       __report_gsfailure         0000000180002a8c f   MSVCRT:gs_report.obj
 0001:00001bd4       __security_init_cookie     0000000180002bd4 f   MSVCRT:gs_support.obj
 0001:00001c80       DllMain                    0000000180002c80 f   MSVCRT:dll_dllmain_stub.obj
 0001:00001ca4       ?__scrt_initialize_type_info@@YAXXZ 0000000180002ca4 f   MSVCRT:tncleanup.obj
 0001:00001cb4       ?__scrt_uninitialize_type_info@@YAXXZ 0000000180002cb4 f   MSVCRT:tncleanup.obj
 0001:00001cc0       __local_stdio_scanf_options 0000000180002cc0 f i MSVCRT:default_local_stdio_options.obj
 0001:00001cc8       __scrt_initialize_default_local_stdio_options 0000000180002cc8 f   MSVCRT:default_local_stdio_options.obj
 0001:00001ce4       __scrt_get_dyn_tls_init_callback 0000000180002ce4 f   MSVCRT:dyn_tls_init.obj
 0001:00001cec       _RTC_Initialize            0000000180002cec f   MSVCRT:initsect.obj
 0001:00001d28       _RTC_Terminate             0000000180002d28 f   MSVCRT:initsect.obj
 0001:00001d64       __isa_available_init       0000000180002d64 f   MSVCRT:cpu_disp.obj
 0001:00001f10       _get_startup_argv_mode     0000000180002f10 f   MSVCRT:argv_mode.obj
 0001:00001f18       __scrt_is_ucrt_dll_in_use  0000000180002f18 f   MSVCRT:ucrt_detection.obj
 0001:00001f30       memset                     0000000180002f30 f   vcruntime:VCRUNTIME140.dll
 0001:00001f36       strstr                     0000000180002f36 f   vcruntime:VCRUNTIME140.dll
 0001:00001f3c       __C_specific_handler       0000000180002f3c f   vcruntime:VCRUNTIME140.dll
 0001:00001f42       __std_type_info_destroy_list 0000000180002f42 f   vcruntime:VCRUNTIME140.dll
 0001:00001f48       strcmp                     0000000180002f48 f   ucrt:api-ms-win-crt-string-l1-1-0.dll
 0001:00001f4e       strlen                     0000000180002f4e f   ucrt:api-ms-win-crt-string-l1-1-0.dll
 0001:00001f54       _initterm                  0000000180002f54 f   ucrt:api-ms-win-crt-runtime-l1-1-0.dll
 0001:00001f5a       _initterm_e                0000000180002f5a f   ucrt:api-ms-win-crt-runtime-l1-1-0.dll
 0001:00001f60       _seh_filter_dll            0000000180002f60 f   ucrt:api-ms-win-crt-runtime-l1-1-0.dll
 0001:00001f66       _configure_narrow_argv     0000000180002f66 f   ucrt:api-ms-win-crt-runtime-l1-1-0.dll
 0001:00001f6c       _initialize_narrow_environment 0000000180002f6c f   ucrt:api-ms-win-crt-runtime-l1-1-0.dll
 0001:00001f72       _initialize_onexit_table   0000000180002f72 f   ucrt:api-ms-win-crt-runtime-l1-1-0.dll
 0001:00001f78       _register_onexit_function  0000000180002f78 f   ucrt:api-ms-win-crt-runtime-l1-1-0.dll
 0001:00001f7e       _execute_onexit_table      0000000180002f7e f   ucrt:api-ms-win-crt-runtime-l1-1-0.dll
 0001:00001f84       _crt_atexit                0000000180002f84 f   ucrt:api-ms-win-crt-runtime-l1-1-0.dll
 0001:00001f8a       _cexit                     0000000180002f8a f   ucrt:api-ms-win-crt-runtime-l1-1-0.dll
 0001:00001f90       __acrt_initialize          0000000180002f90 f   MSVCRT:ucrt_stubs.obj
 0001:00001f90       __acrt_thread_attach       0000000180002f90 f   MSVCRT:ucrt_stubs.obj
 0001:00001f90       __acrt_thread_detach       0000000180002f90 f   MSVCRT:ucrt_stubs.obj
 0001:00001f90       __acrt_uninitialize        0000000180002f90 f   MSVCRT:ucrt_stubs.obj
 0001:00001f90       __acrt_uninitialize_critical 0000000180002f90 f   MSVCRT:ucrt_stubs.obj
 0001:00001f90       __scrt_stub_for_acrt_initialize 0000000180002f90 f   MSVCRT:ucrt_stubs.obj
 0001:00001f90       __scrt_stub_for_acrt_thread_attach 0000000180002f90 f   MSVCRT:ucrt_stubs.obj
 0001:00001f90       __scrt_stub_for_acrt_thread_detach 0000000180002f90 f   MSVCRT:ucrt_stubs.obj
 0001:00001f90       __scrt_stub_for_acrt_uninitialize 0000000180002f90 f   MSVCRT:ucrt_stubs.obj
 0001:00001f90       __scrt_stub_for_acrt_uninitialize_critical 0000000180002f90 f   MSVCRT:ucrt_stubs.obj
 0001:00001f90       __vcrt_initialize          0000000180002f90 f   MSVCRT:ucrt_stubs.obj
 0001:00001f90       __vcrt_thread_attach       0000000180002f90 f   MSVCRT:ucrt_stubs.obj
 0001:00001f90       __vcrt_thread_detach       0000000180002f90 f   MSVCRT:ucrt_stubs.obj
 0001:00001f90       __vcrt_uninitialize        0000000180002f90 f   MSVCRT:ucrt_stubs.obj
 0001:00001f90       __vcrt_uninitialize_critical 0000000180002f90 f   MSVCRT:ucrt_stubs.obj
 0001:00001f94       __scrt_stub_for_is_c_termination_complete 0000000180002f94 f   MSVCRT:ucrt_stubs.obj
 0001:00001f94       _is_c_termination_complete 0000000180002f94 f   MSVCRT:ucrt_stubs.obj
 0001:00001f97       memcpy                     0000000180002f97 f   vcruntime:VCRUNTIME140.dll
 0001:00001fb0       _guard_dispatch_icall_nop  0000000180002fb0 f   MSVCRT:guard_dispatch.obj
 0001:00001fd0       _guard_xfg_dispatch_icall_nop 0000000180002fd0 f   MSVCRT:guard_xfg_dispatch.obj
 0002:00000000       __imp_CloseHandle          0000000180004000     kernel32:KERNEL32.dll
 0002:00000008       __imp_EnterCriticalSection 0000000180004008     kernel32:KERNEL32.dll
 0002:00000010       __imp_LeaveCriticalSection 0000000180004010     kernel32:KERNEL32.dll
 0002:00000018       __imp_InitializeCriticalSectionAndSpinCount 0000000180004018     kernel32:KERNEL32.dll
 0002:00000020       __imp_DeleteCriticalSection 0000000180004020     kernel32:KERNEL32.dll
 0002:00000028       __imp_SetEvent             0000000180004028     kernel32:KERNEL32.dll
 0002:00000030       __imp_ResetEvent           0000000180004030     kernel32:KERNEL32.dll
 0002:00000038       __imp_WaitForSingleObjectEx 0000000180004038     kernel32:KERNEL32.dll
 0002:00000040       __imp_CreateEventW         0000000180004040     kernel32:KERNEL32.dll
 0002:00000048       __imp_GetModuleHandleW     0000000180004048     kernel32:KERNEL32.dll
 0002:00000050       __imp_GetProcAddress       0000000180004050     kernel32:KERNEL32.dll
 0002:00000058       __imp_RtlCaptureContext    0000000180004058     kernel32:KERNEL32.dll
 0002:00000060       __imp_RtlLookupFunctionEntry 0000000180004060     kernel32:KERNEL32.dll
 0002:00000068       __imp_RtlVirtualUnwind     0000000180004068     kernel32:KERNEL32.dll
 0002:00000070       __imp_IsDebuggerPresent    0000000180004070     kernel32:KERNEL32.dll
 0002:00000078       __imp_UnhandledExceptionFilter 0000000180004078     kernel32:KERNEL32.dll
 0002:00000080       __imp_SetUnhandledExceptionFilter 0000000180004080     kernel32:KERNEL32.dll
 0002:00000088       __imp_IsProcessorFeaturePresent 0000000180004088     kernel32:KERNEL32.dll
 0002:00000090       __imp_GetCurrentProcess    0000000180004090     kernel32:KERNEL32.dll
 0002:00000098       __imp_TerminateProcess     0000000180004098     kernel32:KERNEL32.dll
 0002:000000a0       __imp_QueryPerformanceCounter 00000001800040a0     kernel32:KERNEL32.dll
 0002:000000a8       __imp_GetCurrentProcessId  00000001800040a8     kernel32:KERNEL32.dll
 0002:000000b0       __imp_GetCurrentThreadId   00000001800040b0     kernel32:KERNEL32.dll
 0002:000000b8       __imp_GetSystemTimeAsFileTime 00000001800040b8     kernel32:KERNEL32.dll
 0002:000000c0       __imp_DisableThreadLibraryCalls 00000001800040c0     kernel32:KERNEL32.dll
 0002:000000c8       __imp_InitializeSListHead  00000001800040c8     kernel32:KERNEL32.dll
 0002:000000d0       \177KERNEL32_NULL_THUNK_DATA 00000001800040d0     kernel32:KERNEL32.dll
 0002:000000d8       __imp_memset               00000001800040d8     vcruntime:VCRUNTIME140.dll
 0002:000000e0       __imp_strstr               00000001800040e0     vcruntime:VCRUNTIME140.dll
 0002:000000e8       __imp___C_specific_handler 00000001800040e8     vcruntime:VCRUNTIME140.dll
 0002:000000f0       __imp___std_type_info_destroy_list 00000001800040f0     vcruntime:VCRUNTIME140.dll
 0002:000000f8       __imp_memcpy               00000001800040f8     vcruntime:VCRUNTIME140.dll
 0002:00000100       \177VCRUNTIME140_NULL_THUNK_DATA 0000000180004100     vcruntime:VCRUNTIME140.dll
 0002:00000108       __imp__initialize_narrow_environment 0000000180004108     ucrt:api-ms-win-crt-runtime-l1-1-0.dll
 0002:00000110       __imp__cexit               0000000180004110     ucrt:api-ms-win-crt-runtime-l1-1-0.dll
 0002:00000118       __imp__crt_atexit          0000000180004118     ucrt:api-ms-win-crt-runtime-l1-1-0.dll
 0002:00000120       __imp__execute_onexit_table 0000000180004120     ucrt:api-ms-win-crt-runtime-l1-1-0.dll
 0002:00000128       __imp__register_onexit_function 0000000180004128     ucrt:api-ms-win-crt-runtime-l1-1-0.dll
 0002:00000130       __imp__initterm            0000000180004130     ucrt:api-ms-win-crt-runtime-l1-1-0.dll
 0002:00000138       __imp__initterm_e          0000000180004138     ucrt:api-ms-win-crt-runtime-l1-1-0.dll
 0002:00000140       __imp__seh_filter_dll      0000000180004140     ucrt:api-ms-win-crt-runtime-l1-1-0.dll
 0002:00000148       __imp__initialize_onexit_table 0000000180004148     ucrt:api-ms-win-crt-runtime-l1-1-0.dll
 0002:00000150       __imp__configure_narrow_argv 0000000180004150     ucrt:api-ms-win-crt-runtime-l1-1-0.dll
 0002:00000158       \177api-ms-win-crt-runtime-l1-1-0_NULL_THUNK_DATA 0000000180004158     ucrt:api-ms-win-crt-runtime-l1-1-0.dll
 0002:00000160       __imp___acrt_iob_func      0000000180004160     ucrt:api-ms-win-crt-stdio-l1-1-0.dll
 0002:00000168       __imp___stdio_common_vfprintf 0000000180004168     ucrt:api-ms-win-crt-stdio-l1-1-0.dll
 0002:00000170       __imp_fflush               0000000180004170     ucrt:api-ms-win-crt-stdio-l1-1-0.dll
 0002:00000178       \177api-ms-win-crt-stdio-l1-1-0_NULL_THUNK_DATA 0000000180004178     ucrt:api-ms-win-crt-stdio-l1-1-0.dll
 0002:00000180       __imp_strncmp              0000000180004180     ucrt:api-ms-win-crt-string-l1-1-0.dll
 0002:00000188       __imp_strlen               0000000180004188     ucrt:api-ms-win-crt-string-l1-1-0.dll
 0002:00000190       __imp_strncpy              0000000180004190     ucrt:api-ms-win-crt-string-l1-1-0.dll
 0002:00000198       __imp_strcmp               0000000180004198     ucrt:api-ms-win-crt-string-l1-1-0.dll
 0002:000001a0       \177api-ms-win-crt-string-l1-1-0_NULL_THUNK_DATA 00000001800041a0     ucrt:api-ms-win-crt-string-l1-1-0.dll
 0002:000001a8       __guard_check_icall_fptr   00000001800041a8     MSVCRT:guard_support.obj
 0002:000001b0       __guard_xfg_check_icall_fptr 00000001800041b0     MSVCRT:guard_support.obj
 0002:000001b8       __guard_dispatch_icall_fptr 00000001800041b8     MSVCRT:guard_support.obj
 0002:000001c0       __guard_xfg_dispatch_icall_fptr 00000001800041c0     MSVCRT:guard_support.obj
 0002:000001c8       __guard_xfg_table_dispatch_icall_fptr 00000001800041c8     MSVCRT:guard_support.obj
 0002:000001d0       __castguard_check_failure_os_handled_fptr 00000001800041d0     MSVCRT:guard_support.obj
 0002:000001d8       __guard_memcpy_fptr        00000001800041d8     vcruntime:softmemtag.obj
 0002:000001e0       __xc_a                     00000001800041e0     MSVCRT:initializers.obj
 0002:000001e8       __xc_z                     00000001800041e8     MSVCRT:initializers.obj
 0002:000001f0       __xi_a                     00000001800041f0     MSVCRT:initializers.obj
 0002:00000200       __xi_z                     0000000180004200     MSVCRT:initializers.obj
 0002:00000208       __xl_a                     0000000180004208     MSVCRT:tlssup.obj
 0002:00000210       __xl_z                     0000000180004210     MSVCRT:tlssup.obj
 0002:00000218       __xp_a                     0000000180004218     MSVCRT:initializers.obj
 0002:00000220       __xp_z                     0000000180004220     MSVCRT:initializers.obj
 0002:00000228       __xt_a                     0000000180004228     MSVCRT:initializers.obj
 0002:00000230       __xt_z                     0000000180004230     MSVCRT:initializers.obj
 0002:00000240       ??_C@_0BK@OLPKINJM@Lgetstacktr06$TestThread?$DL@ 0000000180004240     libgetstacktr06.obj
 0002:0000025c       ??_C@_06CHHFAIGH@chain4@   000000018000425c     libgetstacktr06.obj
 0002:00000264       ??_C@_03GAEACAIP@?$CI?$CJV@ 0000000180004264     libgetstacktr06.obj
 0002:00000268       ??_C@_06GIDEJOKA@chain3@   0000000180004268     libgetstacktr06.obj
 0002:00000270       ??_C@_06HBCPKPOB@chain2@   0000000180004270     libgetstacktr06.obj
 0002:00000278       ??_C@_06FKACPMCC@chain1@   0000000180004278     libgetstacktr06.obj
 0002:00000280       ??_C@_03LGMJKEGG@run@      0000000180004280     libgetstacktr06.obj
 0002:00000288       ??_C@_0BD@KAGNMIPJ@Ljava?1lang?1Thread?$DL@ 0000000180004288     libgetstacktr06.obj
 0002:000002a0       ??_C@_07MKMHKNKM@runWith@  00000001800042a0     libgetstacktr06.obj
 0002:000002a8       ??_C@_0CK@FDNODPMG@?$CILjava?1lang?1Object?$DLLjava?1lang?1R@ 00000001800042a8     libgetstacktr06.obj
 0002:000002d8       ??_C@_0BK@OCGOFPAH@Ljava?1lang?1VirtualThread?$DL@ 00000001800042d8     libgetstacktr06.obj
 0002:000002f8       ??_C@_0BI@HFKLNKLF@?$CILjava?1lang?1Runnable?$DL?$CJV@ 00000001800042f8     libgetstacktr06.obj
 0002:00000310       ??_C@_0CO@DMNLHMPC@Ljava?1lang?1VirtualThread$VThrea@ 0000000180004310     libgetstacktr06.obj
 0002:00000340       ??_C@_0N@MKJNEODC@lambda$new$0@ 0000000180004340     libgetstacktr06.obj
 0002:00000350       ??_C@_0DB@MLKGFMPP@?$CILjava?1lang?1VirtualThread?$DLLjava@ 0000000180004350     libgetstacktr06.obj
 0002:00000388       ??_C@_0DG@EGJOJPOI@Ljava?1lang?1VirtualThread$VThrea@ 0000000180004388     libgetstacktr06.obj
 0002:000003c0       ??_C@_0BP@EGNIICBH@Ljdk?1internal?1vm?1Continuation?$DL@ 00000001800043c0     libgetstacktr06.obj
 0002:000003e0       ??_C@_06BHKOGBK@enter0@    00000001800043e0     libgetstacktr06.obj
 0002:000003e8       ??_C@_05IHEOCMON@enter@    00000001800043e8     libgetstacktr06.obj
 0002:000003f0       ??_C@_0CD@PKCBGPGJ@?$CILjdk?1internal?1vm?1Continuation?$DL@ 00000001800043f0     libgetstacktr06.obj
 0002:00000418       ??_C@_0DM@KLJPMIDM@check_jvmti_status?3?5JVMTI?5funct@ 0000000180004418     libgetstacktr06.obj
 0002:00000458       ??_C@_0CL@MEELKAEL@deallocate?3?5error?5in?5JVMTI?5Deal@ 0000000180004458     libgetstacktr06.obj
 0002:00000488       ??_C@_0DO@CNKPCOHC@get_method_class_name?3?5error?5in@ 0000000180004488     libgetstacktr06.obj
 0002:000004c8       ??_C@_0DI@ODOBMANA@get_method_class_name?3?5error?5in@ 00000001800044c8     libgetstacktr06.obj
 0002:00000500       ??_C@_0CP@IBPBEBM@get_method_class_name?3?5error?5in@ 0000000180004500     libgetstacktr06.obj
 0002:00000530       ??_C@_0CL@BDMIAND@print_method?3?5error?5in?5JVMTI?5Ge@ 0000000180004530     libgetstacktr06.obj
 0002:00000560       ??_C@_0P@GFDDDNG@?$CF2d?3?5?$CFs?3?5?$CFs?$CFs?6@ 0000000180004560     libgetstacktr06.obj
 0002:00000570       ??_C@_01EEMJAFIK@?6@       0000000180004570     libgetstacktr06.obj
 0002:00000578       ??_C@_0BB@NEONAMMP@?$DMUnnamed?5thread?$DO@ 0000000180004578     libgetstacktr06.obj
 0002:00000590       ??_C@_0DD@PEIMAGBL@get_thread_name?3?5error?5in?5JVMTI@ 0000000180004590     libgetstacktr06.obj
 0002:000005c8       ??_C@_0BC@KKCEBIKL@GetClassSignature@ 00000001800045c8     libgetstacktr06.obj
 0002:000005e0       ??_C@_0DA@DGJBBBMN@print_stack_trace?3?5error?5in?5JVM@ 00000001800045e0     libgetstacktr06.obj
 0002:00000610       ??_C@_0DC@EJGPEKOE@JVMTI?5Stack?5Trace?5for?5thread?5?$CFs@ 0000000180004610     libgetstacktr06.obj
 0002:00000648       ??_C@_0BB@JCNMKLLK@JVMTI_ERROR_NONE@ 0000000180004648     libgetstacktr06.obj
 0002:00000660       ??_C@_0BL@LDIMKLPH@JVMTI_ERROR_INVALID_THREAD@ 0000000180004660     libgetstacktr06.obj
 0002:00000680       ??_C@_0CB@PJFPAIKJ@JVMTI_ERROR_INVALID_THREAD_GROU@ 0000000180004680     libgetstacktr06.obj
 0002:000006a8       ??_C@_0BN@LLMKHMNF@JVMTI_ERROR_INVALID_PRIORITY@ 00000001800046a8     libgetstacktr06.obj
 0002:000006c8       ??_C@_0CB@MBOFKAGB@JVMTI_ERROR_THREAD_NOT_SUSPENDE@ 00000001800046c8     libgetstacktr06.obj
 0002:000006f0       ??_C@_0BN@FABOLPBI@JVMTI_ERROR_THREAD_SUSPENDED@ 00000001800046f0     libgetstacktr06.obj
 0002:00000710       ??_C@_0BN@FDGNOBJM@JVMTI_ERROR_THREAD_NOT_ALIVE@ 0000000180004710     libgetstacktr06.obj
 0002:00000730       ??_C@_0BL@GOBIFKNJ@JVMTI_ERROR_INVALID_OBJECT@ 0000000180004730     libgetstacktr06.obj
 0002:00000750       ??_C@_0BK@FCMAJPPC@JVMTI_ERROR_INVALID_CLASS@ 0000000180004750     libgetstacktr06.obj
 0002:00000770       ??_C@_0BP@IKLLBKEB@JVMTI_ERROR_CLASS_NOT_PREPARED@ 0000000180004770     libgetstacktr06.obj
 0002:00000790       ??_C@_0BN@KLPPLKG@JVMTI_ERROR_INVALID_METHODID@ 0000000180004790     libgetstacktr06.obj
 0002:000007b0       ??_C@_0BN@BCEKOKND@JVMTI_ERROR_INVALID_LOCATION@ 00000001800047b0     libgetstacktr06.obj
 0002:000007d0       ??_C@_0BM@DFDGPME@JVMTI_ERROR_INVALID_FIELDID@ 00000001800047d0     libgetstacktr06.obj
 0002:000007f0       ??_C@_0BL@NELIEPEC@JVMTI_ERROR_NO_MORE_FRAMES@ 00000001800047f0     libgetstacktr06.obj
 0002:00000810       ??_C@_0BJ@BDBECFDM@JVMTI_ERROR_OPAQUE_FRAME@ 0000000180004810     libgetstacktr06.obj
 0002:00000830       ??_C@_0BK@MIIFNLOB@JVMTI_ERROR_TYPE_MISMATCH@ 0000000180004830     libgetstacktr06.obj
 0002:00000850       ??_C@_0BJ@HPCAOILC@JVMTI_ERROR_INVALID_SLOT@ 0000000180004850     libgetstacktr06.obj
 0002:00000870       ??_C@_0BG@CHILOPNI@JVMTI_ERROR_DUPLICATE@ 0000000180004870     libgetstacktr06.obj
 0002:00000888       ??_C@_0BG@DIEMLHKM@JVMTI_ERROR_NOT_FOUND@ 0000000180004888     libgetstacktr06.obj
 0002:000008a0       ??_C@_0BM@NHMCKHOB@JVMTI_ERROR_INVALID_MONITOR@ 00000001800048a0     libgetstacktr06.obj
 0002:000008c0       ??_C@_0BO@PPEDAJGL@JVMTI_ERROR_NOT_MONITOR_OWNER@ 00000001800048c0     libgetstacktr06.obj
 0002:000008e0       ??_C@_0BG@FCAIPEID@JVMTI_ERROR_INTERRUPT@ 00000001800048e0     libgetstacktr06.obj
 0002:000008f8       ??_C@_0CB@EGDBNKOI@JVMTI_ERROR_INVALID_CLASS_FORMA@ 00000001800048f8     libgetstacktr06.obj
 0002:00000920       ??_C@_0CG@DGKOGIAL@JVMTI_ERROR_CIRCULAR_CLASS_DEFI@ 0000000180004920     libgetstacktr06.obj
 0002:00000948       ??_C@_0BP@ICEALPKC@JVMTI_ERROR_FAILS_VERIFICATION@ 0000000180004948     libgetstacktr06.obj
 0002:00000968       ??_C@_0DC@JDACLMIO@JVMTI_ERROR_UNSUPPORTED_REDEFIN@ 0000000180004968     libgetstacktr06.obj
 0002:000009a0       ??_C@_0DE@GKDKNOMJ@JVMTI_ERROR_UNSUPPORTED_REDEFIN@ 00000001800049a0     libgetstacktr06.obj
 0002:000009d8       ??_C@_0BO@LAFKIOG@JVMTI_ERROR_INVALID_TYPESTATE@ 00000001800049d8     libgetstacktr06.obj
 0002:000009f8       ??_C@_0DH@INDGCLLB@JVMTI_ERROR_UNSUPPORTED_REDEFIN@ 00000001800049f8     libgetstacktr06.obj
 0002:00000a30       ??_C@_0DE@NHEOMMGI@JVMTI_ERROR_UNSUPPORTED_REDEFIN@ 0000000180004a30     libgetstacktr06.obj
 0002:00000a68       ??_C@_0CA@EKPNJOEP@JVMTI_ERROR_UNSUPPORTED_VERSION@ 0000000180004a68     libgetstacktr06.obj
 0002:00000a88       ??_C@_0BN@OFFMAHHL@JVMTI_ERROR_NAMES_DONT_MATCH@ 0000000180004a88     libgetstacktr06.obj
 0002:00000aa8       ??_C@_0DN@HHBBLAKE@JVMTI_ERROR_UNSUPPORTED_REDEFIN@ 0000000180004aa8     libgetstacktr06.obj
 0002:00000ae8       ??_C@_0DO@HMBGBGNA@JVMTI_ERROR_UNSUPPORTED_REDEFIN@ 0000000180004ae8     libgetstacktr06.obj
 0002:00000b28       ??_C@_0BP@PBECGKHJ@JVMTI_ERROR_UNMODIFIABLE_CLASS@ 0000000180004b28     libgetstacktr06.obj
 0002:00000b48       ??_C@_0BK@CANILEHF@JVMTI_ERROR_NOT_AVAILABLE@ 0000000180004b48     libgetstacktr06.obj
 0002:00000b68       ??_C@_0CE@INJKMEFK@JVMTI_ERROR_MUST_POSSESS_CAPABI@ 0000000180004b68     libgetstacktr06.obj
 0002:00000b90       ??_C@_0BJ@LBFPFPDM@JVMTI_ERROR_NULL_POINTER@ 0000000180004b90     libgetstacktr06.obj
 0002:00000bb0       ??_C@_0BP@CHJPNNEM@JVMTI_ERROR_ABSENT_INFORMATION@ 0000000180004bb0     libgetstacktr06.obj
 0002:00000bd0       ??_C@_0BP@OMFMNLC@JVMTI_ERROR_INVALID_EVENT_TYPE@ 0000000180004bd0     libgetstacktr06.obj
 0002:00000bf0       ??_C@_0BN@BIBNPHHO@JVMTI_ERROR_ILLEGAL_ARGUMENT@ 0000000180004bf0     libgetstacktr06.obj
 0002:00000c10       ??_C@_0BK@KKNDHDCE@JVMTI_ERROR_NATIVE_METHOD@ 0000000180004c10     libgetstacktr06.obj
 0002:00000c30       ??_C@_0BK@PMKCFHAE@JVMTI_ERROR_OUT_OF_MEMORY@ 0000000180004c30     libgetstacktr06.obj
 0002:00000c50       ??_C@_0BK@NNJBDMNB@JVMTI_ERROR_ACCESS_DENIED@ 0000000180004c50     libgetstacktr06.obj
 0002:00000c70       ??_C@_0BI@GHECLMNC@JVMTI_ERROR_WRONG_PHASE@ 0000000180004c70     libgetstacktr06.obj
 0002:00000c88       ??_C@_0BF@OLIHJOII@JVMTI_ERROR_INTERNAL@ 0000000180004c88     libgetstacktr06.obj
 0002:00000ca0       ??_C@_0BO@EOHGKJHI@JVMTI_ERROR_UNATTACHED_THREAD@ 0000000180004ca0     libgetstacktr06.obj
 0002:00000cc0       ??_C@_0CA@LKHFDACL@JVMTI_ERROR_INVALID_ENVIRONMENT@ 0000000180004cc0     libgetstacktr06.obj
 0002:00000ce0       ??_C@_0BA@MMFHLOKK@?$DMunknown?5error?$DO@ 0000000180004ce0     libgetstacktr06.obj
 0002:00000cf0       ??_C@_0FC@DIHHIAJG@jvmti_common?5set_event_notifica@ 0000000180004cf0     libgetstacktr06.obj
 0002:00000d48       ??_C@_0CD@GMCIPOPD@Calling?5compare_stack_trace?5for@ 0000000180004d48     libgetstacktr06.obj
 0002:00000d70       ??_C@_0BG@PLBEAPMH@GetStackTrace?5failed?4@ 0000000180004d70     libgetstacktr06.obj
 0002:00000d88       ??_C@_0CE@BOIEBIDC@Number?5of?5frames?3?5?$CFd?0?5expected?3@ 0000000180004d88     libgetstacktr06.obj
 0002:00000db0       ??_C@_0DJ@LEGDJKLJ@Number?5of?5expected_frames?3?5?$CFd?5i@ 0000000180004db0     libgetstacktr06.obj
 0002:00000df0       ??_C@_0BL@BGCNDIFA@?$DO?$DO?$DO?5checking?5frame?$CD?$CFd?5?4?4?4?6@ 0000000180004df0     libgetstacktr06.obj
 0002:00000e10       ??_C@_0CA@BBPGJIJK@GetMethodDeclaringClass?5failed?4@ 0000000180004e10     libgetstacktr06.obj
 0002:00000e30       ??_C@_0O@GILEHKFL@GetMethodName@ 0000000180004e30     libgetstacktr06.obj
 0002:00000e40       ??_C@_0BE@LCEDINOL@?$DO?$DO?$DO?5?5?5class?3?5?5?$CC?$CFs?$CC?6@ 0000000180004e40     libgetstacktr06.obj
 0002:00000e58       ??_C@_0BG@LPMLMDDJ@?$DO?$DO?$DO?5?5?5method?3?5?$CC?$CFs?$CFs?$CC?6@ 0000000180004e58     libgetstacktr06.obj
 0002:00000e70       ??_C@_0BD@BILODKNO@?$DO?$DO?$DO?5?5?5?$CFd?5?4?4?4?5done?6@ 0000000180004e70     libgetstacktr06.obj
 0002:00000e88       ??_C@_0BB@EIDHBFAC@expected?5idx?5?$CFd?6@ 0000000180004e88     libgetstacktr06.obj
 0002:00000ea0       ??_C@_08DIGBCCMO@$$Lambda@ 0000000180004ea0     libgetstacktr06.obj
 0002:00000eb0       ??_C@_0CO@DLOKDPGM@Comparing?5only?5first?5?$CFzu?5chars?5@ 0000000180004eb0     libgetstacktr06.obj
 0002:00000ee0       ??_C@_0DC@EBCCBDLN@?$CIframe?$CD?$CFd?$CJ?5wrong?5class?5sig?3?5?$CC?$CFs@ 0000000180004ee0     libgetstacktr06.obj
 0002:00000f18       ??_C@_0DE@GEDGABNF@?$CIframe?$CD?$CFd?$CJ?5wrong?5method?5name?3?5?$CC@ 0000000180004f18     libgetstacktr06.obj
 0002:00000f50       ??_C@_0DD@OBLJKHIF@?$CIframe?$CD?$CFd?$CJ?5wrong?5method?5sig?3?5?$CC?$CF@ 0000000180004f50     libgetstacktr06.obj
 0002:00000f88       ??_C@_0CM@EGMIFBJC@ERROR?3?5didn?8t?5know?5where?5we?5got@ 0000000180004f88     libgetstacktr06.obj
 0002:00000fb8       ??_C@_0BI@KFICPHJJ@ClearBreakpoint?5failed?4@ 0000000180004fb8     libgetstacktr06.obj
 0002:00000fd0       ??_C@_0BH@DEEEBFCO@?$DO?$DO?$DO?5popping?5frame?5?4?4?4?6@ 0000000180004fd0     libgetstacktr06.obj
 0002:00000fe8       ??_C@_0BA@CJINCHKC@PopFrame?5failed@ 0000000180004fe8     libgetstacktr06.obj
 0002:00000ff8       ??_C@_0CC@HGEBPIBI@Stacktrace?5differs?5from?5expecte@ 0000000180004ff8     libgetstacktr06.obj
 0002:00001020       ??_C@_0BL@IONOAEOO@java?1lang?1RuntimeException@ 0000000180005020     libgetstacktr06.obj
 0002:00001040       ??_C@_0CJ@KCDEKOCJ@Wrong?5result?5of?5a?5valid?5call?5to@ 0000000180005040     libgetstacktr06.obj
 0002:00001070       ??_C@_0CN@LKPEOJPO@?$CIAddCapabilities?$CJ?5unexpected?5er@ 0000000180005070     libgetstacktr06.obj
 0002:000010a0       ??_C@_0CN@BCCBOHCH@?$CIGetCapabilities?$CJ?5unexpected?5er@ 00000001800050a0     libgetstacktr06.obj
 0002:000010d0       ??_C@_0CP@IMINGNLL@?$CISetEventCallbacks?$CJ?5unexpected?5@ 00000001800050d0     libgetstacktr06.obj
 0002:00001100       ??_C@_0L@GIHILDI@checkPoint@ 0000000180005100     libgetstacktr06.obj
 0002:00001110       ??_C@_0CN@GIADEMBI@Cannot?5find?5Method?5ID?5for?5metho@ 0000000180005110     libgetstacktr06.obj
 0002:00001140       ??_C@_0BG@BCCBDDLF@SetBreakpoint?5failed?4@ 0000000180005140     libgetstacktr06.obj
 0002:00001160       ??_C@_1EC@JIJBPKFM@?$AAa?$AAp?$AAi?$AA?9?$AAm?$AAs?$AA?9?$AAw?$AAi?$AAn?$AA?9?$AAc?$AAo?$AAr?$AAe@ 0000000180005160     MSVCRT:thread_safe_statics.obj
 0002:000011a8       ??_C@_1BK@MGMFAEKH@?$AAk?$AAe?$AAr?$AAn?$AAe?$AAl?$AA3?$AA2?$AA?4?$AAd?$AAl?$AAl@ 00000001800051a8     MSVCRT:thread_safe_statics.obj
 0002:000011c8       ??_C@_0BJ@JEBJOJFJ@SleepConditionVariableCS@ 00000001800051c8     MSVCRT:thread_safe_statics.obj
 0002:000011e8       ??_C@_0BJ@PGPPEPCC@WakeAllConditionVariable@ 00000001800051e8     MSVCRT:thread_safe_statics.obj
 0002:00001208       _pDefaultRawDllMain        0000000180005208     MSVCRT:dll_dllmain.obj
 0002:00001208       _pRawDllMain               0000000180005208     MSVCRT:dll_dllmain.obj
 0002:00001210       __xmm@ffffffffffffffffffffffffffffffff 0000000180005210     MSVCRT:utility.obj
 0002:00001230       _load_config_used          0000000180005230     MSVCRT:loadcfg.obj
 0002:00001400       _tls_used                  0000000180005400     MSVCRT:tlssup.obj
 0002:00001428       __volatile_metadata        0000000180005428     <linker-defined>
 0002:000017a8       __rtc_iaa                  00000001800057a8     MSVCRT:initsect.obj
 0002:000017b0       __rtc_izz                  00000001800057b0     MSVCRT:initsect.obj
 0002:000017b8       __rtc_taa                  00000001800057b8     MSVCRT:initsect.obj
 0002:000017c0       __rtc_tzz                  00000001800057c0     MSVCRT:initsect.obj
 0002:000017c8       _tls_start                 00000001800057c8     MSVCRT:tlssup.obj
 0002:000017cc       _Init_thread_epoch         00000001800057cc     MSVCRT:thread_safe_statics.obj
 0002:000017d0       _tls_end                   00000001800057d0     MSVCRT:tlssup.obj
 0002:00001a78       __IMPORT_DESCRIPTOR_KERNEL32 0000000180005a78     kernel32:KERNEL32.dll
 0002:00001a8c       __IMPORT_DESCRIPTOR_VCRUNTIME140 0000000180005a8c     vcruntime:VCRUNTIME140.dll
 0002:00001aa0       __IMPORT_DESCRIPTOR_api-ms-win-crt-stdio-l1-1-0 0000000180005aa0     ucrt:api-ms-win-crt-stdio-l1-1-0.dll
 0002:00001ab4       __IMPORT_DESCRIPTOR_api-ms-win-crt-string-l1-1-0 0000000180005ab4     ucrt:api-ms-win-crt-string-l1-1-0.dll
 0002:00001ac8       __IMPORT_DESCRIPTOR_api-ms-win-crt-runtime-l1-1-0 0000000180005ac8     ucrt:api-ms-win-crt-runtime-l1-1-0.dll
 0002:00001adc       __NULL_IMPORT_DESCRIPTOR   0000000180005adc     kernel32:KERNEL32.dll
 0003:000001c8       _Init_global_epoch         00000001800071c8     MSVCRT:thread_safe_statics.obj
 0003:000001d0       __security_cookie          00000001800071d0     MSVCRT:gs_cookie.obj
 0003:000001d8       __security_cookie_complement 00000001800071d8     MSVCRT:gs_cookie.obj
 0003:000001e0       __scrt_native_dllmain_reason 00000001800071e0     MSVCRT:utility.obj
 0003:000001e8       __isa_available            00000001800071e8     MSVCRT:cpu_disp.obj
 0003:000001ec       __isa_enabled              00000001800071ec     MSVCRT:cpu_disp.obj
 0003:000001f0       __memset_fast_string_threshold 00000001800071f0     MSVCRT:cpu_disp.obj
 0003:000001f8       __memset_nt_threshold      00000001800071f8     MSVCRT:cpu_disp.obj
 0003:00000200       __scrt_ucrt_dll_is_in_use  0000000180007200     MSVCRT:ucrt_stubs.obj
 0003:00000210       ?_OptionsStorage@?1??__local_stdio_printf_options@@9@4_KA 0000000180007210     libgetstacktr06.obj
 0003:000003c0       _tls_index                 00000001800073c0     MSVCRT:tlssup.obj
 0003:000003c8       __scrt_current_native_startup_state 00000001800073c8     MSVCRT:utility.obj
 0003:000003d0       __scrt_native_startup_lock 00000001800073d0     MSVCRT:utility.obj
 0003:00000410       __scrt_debugger_hook_flag  0000000180007410     MSVCRT:utility_desktop.obj
 0003:00000990       ?__type_info_root_node@@3U__type_info_node@@A 0000000180007990     MSVCRT:tncleanup.obj
 0003:000009a0       ?_OptionsStorage@?1??__local_stdio_scanf_options@@9@4_KA 00000001800079a0     MSVCRT:default_local_stdio_options.obj
 0003:000009a8       __favor                    00000001800079a8     MSVCRT:cpu_disp.obj
 0003:000009b0       __dyn_tls_init_callback    00000001800079b0     <common>

 entry point at        0001:00001540

 Static symbols

 0000:ffff6000       .debug$S                   0000000180000000     getstacktr06.exp
 0000:ffff6000       .debug$S                   0000000180000000     vcruntime:VCRUNTIME140.dll
 0000:ffff6000       .debug$S                   0000000180000000     vcruntime:VCRUNTIME140.dll
 0000:ffff6000       .debug$S                   0000000180000000     vcruntime:VCRUNTIME140.dll
 0000:ffff6000       .debug$S                   0000000180000000     vcruntime:VCRUNTIME140.dll
 0000:ffff6000       .debug$S                   0000000180000000     vcruntime:VCRUNTIME140.dll
 0000:ffff6000       .debug$S                   0000000180000000     vcruntime:VCRUNTIME140.dll
 0000:ffff6000       .debug$S                   0000000180000000     vcruntime:VCRUNTIME140.dll
 0000:ffff6000       .debug$S                   0000000180000000     ucrt:api-ms-win-crt-runtime-l1-1-0.dll
 0000:ffff6000       .debug$S                   0000000180000000     ucrt:api-ms-win-crt-runtime-l1-1-0.dll
 0000:ffff6000       .debug$S                   0000000180000000     ucrt:api-ms-win-crt-runtime-l1-1-0.dll
 0000:ffff6000       .debug$S                   0000000180000000     ucrt:api-ms-win-crt-runtime-l1-1-0.dll
 0000:ffff6000       .debug$S                   0000000180000000     ucrt:api-ms-win-crt-runtime-l1-1-0.dll
 0000:ffff6000       .debug$S                   0000000180000000     ucrt:api-ms-win-crt-runtime-l1-1-0.dll
 0000:ffff6000       .debug$S                   0000000180000000     ucrt:api-ms-win-crt-runtime-l1-1-0.dll
 0000:ffff6000       .debug$S                   0000000180000000     ucrt:api-ms-win-crt-runtime-l1-1-0.dll
 0000:ffff6000       .debug$S                   0000000180000000     ucrt:api-ms-win-crt-runtime-l1-1-0.dll
 0000:ffff6000       .debug$S                   0000000180000000     ucrt:api-ms-win-crt-runtime-l1-1-0.dll
 0000:ffff6000       .debug$S                   0000000180000000     ucrt:api-ms-win-crt-runtime-l1-1-0.dll
 0000:ffff6000       .debug$S                   0000000180000000     ucrt:api-ms-win-crt-runtime-l1-1-0.dll
 0000:ffff6000       .debug$S                   0000000180000000     ucrt:api-ms-win-crt-stdio-l1-1-0.dll
 0000:ffff6000       .debug$S                   0000000180000000     ucrt:api-ms-win-crt-stdio-l1-1-0.dll
 0000:ffff6000       .debug$S                   0000000180000000     ucrt:api-ms-win-crt-stdio-l1-1-0.dll
 0000:ffff6000       .debug$S                   0000000180000000     ucrt:api-ms-win-crt-string-l1-1-0.dll
 0000:ffff6000       .debug$S                   0000000180000000     ucrt:api-ms-win-crt-string-l1-1-0.dll
 0000:ffff6000       .debug$S                   0000000180000000     ucrt:api-ms-win-crt-string-l1-1-0.dll
 0000:ffff6000       .debug$S                   0000000180000000     ucrt:api-ms-win-crt-string-l1-1-0.dll
 0000:ffff6000       .debug$S                   0000000180000000     ucrt:api-ms-win-crt-string-l1-1-0.dll
 0000:ffff6000       .debug$S                   0000000180000000     kernel32:KERNEL32.dll
 0000:ffff6000       .debug$S                   0000000180000000     kernel32:KERNEL32.dll
 0000:ffff6000       .debug$S                   0000000180000000     kernel32:KERNEL32.dll
 0000:ffff6000       .debug$S                   0000000180000000     kernel32:KERNEL32.dll
 0000:ffff6000       .debug$S                   0000000180000000     kernel32:KERNEL32.dll
 0000:ffff6000       .debug$S                   0000000180000000     kernel32:KERNEL32.dll
 0000:ffff6000       .debug$S                   0000000180000000     kernel32:KERNEL32.dll
 0000:ffff6000       .debug$S                   0000000180000000     kernel32:KERNEL32.dll
 0000:ffff6000       .debug$S                   0000000180000000     kernel32:KERNEL32.dll
 0000:ffff6000       .debug$S                   0000000180000000     kernel32:KERNEL32.dll
 0000:ffff6000       .debug$S                   0000000180000000     kernel32:KERNEL32.dll
 0000:ffff6000       .debug$S                   0000000180000000     kernel32:KERNEL32.dll
 0000:ffff6000       .debug$S                   0000000180000000     kernel32:KERNEL32.dll
 0000:ffff6000       .debug$S                   0000000180000000     kernel32:KERNEL32.dll
 0000:ffff6000       .debug$S                   0000000180000000     kernel32:KERNEL32.dll
 0000:ffff6000       .debug$S                   0000000180000000     kernel32:KERNEL32.dll
 0000:ffff6000       .debug$S                   0000000180000000     kernel32:KERNEL32.dll
 0000:ffff6000       .debug$S                   0000000180000000     kernel32:KERNEL32.dll
 0000:ffff6000       .debug$S                   0000000180000000     kernel32:KERNEL32.dll
 0000:ffff6000       .debug$S                   0000000180000000     kernel32:KERNEL32.dll
 0000:ffff6000       .debug$S                   0000000180000000     kernel32:KERNEL32.dll
 0000:ffff6000       .debug$S                   0000000180000000     kernel32:KERNEL32.dll
 0000:ffff6000       .debug$S                   0000000180000000     kernel32:KERNEL32.dll
 0000:ffff6000       .debug$S                   0000000180000000     kernel32:KERNEL32.dll
 0000:ffff6000       .debug$S                   0000000180000000     kernel32:KERNEL32.dll
 0000:ffff6000       .debug$S                   0000000180000000     kernel32:KERNEL32.dll
 0000:ffff6000       .debug$S                   0000000180000000     kernel32:KERNEL32.dll
 0000:ffff6000       .debug$S                   0000000180000000     kernel32:KERNEL32.dll
 0001:000002c4       ?check_jvmti_status@@YAXPEAUJNIEnv_@@W4jvmtiError@@PEBD@Z 00000001800012c4 f   libgetstacktr06.obj
 0001:00000678       ?print_method@@YAXPEAU_jvmtiEnv@@PEAUJNIEnv_@@PEAU_jmethodID@@H@Z 0000000180001678 f   libgetstacktr06.obj
 0001:00000870       ?print_stack_trace@@YAXPEAU_jvmtiEnv@@PEAUJNIEnv_@@PEAV_jobject@@@Z 0000000180001870 f   libgetstacktr06.obj
 0001:00000f00       ?__scrt_initialize_thread_safe_statics@@YAHXZ 0000000180001f00 f   MSVCRT:thread_safe_statics.obj
 0001:00000fd0       ?__scrt_uninitialize_thread_safe_statics@@YAXXZ 0000000180001fd0 f   MSVCRT:thread_safe_statics.obj
 0001:000011f0       $$000000                   00000001800021f0     MSVCRT:amdsecgs.obj
 0001:00001220       ?dllmain_crt_dispatch@@YAHQEAUHINSTANCE__@@KQEAX@Z 0000000180002220 f   MSVCRT:dll_dllmain.obj
 0001:00001270       ?dllmain_crt_process_attach@@YAHQEAUHINSTANCE__@@QEAX@Z 0000000180002270 f   MSVCRT:dll_dllmain.obj
 0001:00001388       ?dllmain_crt_process_detach@@YAH_N@Z 0000000180002388 f   MSVCRT:dll_dllmain.obj
 0001:0000140c       ?dllmain_dispatch@@YAHQEAUHINSTANCE__@@KQEAX@Z 000000018000240c f   MSVCRT:dll_dllmain.obj
 0001:00001b60       capture_previous_context   0000000180002b60 f   MSVCRT:gs_report.obj
 0001:00001fa0       $$000000                   0000000180002fa0     MSVCRT:guard_dispatch.obj
 0001:00001fc0       $$000000                   0000000180002fc0     MSVCRT:guard_xfg_dispatch.obj
 0001:00001fd6       ?fin$0@?0??dllmain_crt_process_attach@@YAHQEAUHINSTANCE__@@QEAX@Z@4HA 0000000180002fd6 f   MSVCRT:dll_dllmain.obj
 0001:00001fed       ?fin$0@?0??dllmain_crt_process_detach@@YAH_N@Z@4HA 0000000180002fed f   MSVCRT:dll_dllmain.obj
 0001:00002006       ?fin$1@?0??dllmain_crt_process_detach@@YAH_N@Z@4HA 0000000180003006 f   MSVCRT:dll_dllmain.obj
 0001:0000201a       ?filt$0@?0??dllmain_dispatch@@YAHQEAUHINSTANCE__@@KQEAX@Z@4HA 000000018000301a f   MSVCRT:dll_dllmain.obj
 0001:00002050       __scrt_is_nonwritable_in_current_image$filt$0 0000000180003050 f   MSVCRT:utility.obj
 0002:000001f8       ?__scrt_initialize_tss_var@@3P6AHXZEA 00000001800041f8     MSVCRT:thread_safe_statics.obj
 0002:00001220       GS_ExceptionPointers       0000000180005220     MSVCRT:gs_report.obj
 0002:000017d8       $unwind$printf             00000001800057d8     libgetstacktr06.obj
 0002:000017e4       $unwind$Agent_OnLoad       00000001800057e4     libgetstacktr06.obj
 0002:000017f4       $unwind$?check_jvmti_status@@YAXPEAUJNIEnv_@@W4jvmtiError@@PEBD@Z 00000001800057f4     libgetstacktr06.obj
 0002:00001804       $unwind$?print_method@@YAXPEAU_jvmtiEnv@@PEAUJNIEnv_@@PEAU_jmethodID@@H@Z 0000000180005804     libgetstacktr06.obj
 0002:0000181c       $unwind$?print_stack_trace@@YAXPEAU_jvmtiEnv@@PEAUJNIEnv_@@PEAV_jobject@@@Z 000000018000581c     libgetstacktr06.obj
 0002:0000183c       $unwind$?compare_stack_trace@@YAHPEAU_jvmtiEnv@@PEAUJNIEnv_@@PEAV_jobject@@QEAUframe_info@@HH@Z 000000018000583c     libgetstacktr06.obj
 0002:0000185c       $unwind$Breakpoint         000000018000585c     libgetstacktr06.obj
 0002:0000185c       $unwind$_RTC_Initialize    000000018000585c     MSVCRT:initsect.obj
 0002:0000185c       $unwind$_RTC_Terminate     000000018000585c     MSVCRT:initsect.obj
 0002:0000185c       $unwind$?__scrt_initialize_thread_safe_statics@@YAHXZ 000000018000585c     MSVCRT:thread_safe_statics.obj
 0002:00001868       $unwind$SingleStep         0000000180005868     libgetstacktr06.obj
 0002:0000187c       $unwind$Java_getstacktr06_getReady 000000018000587c     libgetstacktr06.obj
 0002:0000187c       $unwind$__raise_securityfailure 000000018000587c     MSVCRT:gs_report.obj
 0002:0000187c       $unwind$_Init_thread_footer 000000018000587c     MSVCRT:thread_safe_statics.obj
 0002:0000187c       $unwind$_Init_thread_header 000000018000587c     MSVCRT:thread_safe_statics.obj
 0002:0000187c       $unwind$_Init_thread_wait  000000018000587c     MSVCRT:thread_safe_statics.obj
 0002:0000187c       $unwind$__scrt_initialize_crt 000000018000587c     MSVCRT:utility.obj
 0002:0000187c       $unwind$__scrt_initialize_onexit_tables 000000018000587c     MSVCRT:utility.obj
 0002:0000187c       $unwind$__scrt_release_startup_lock 000000018000587c     MSVCRT:utility.obj
 0002:0000187c       $unwind$__scrt_uninitialize_crt 000000018000587c     MSVCRT:utility.obj
 0002:0000187c       $unwind$_onexit            000000018000587c     MSVCRT:utility.obj
 0002:00001884       $unwind$__scrt_initialize_default_local_stdio_options 0000000180005884     MSVCRT:default_local_stdio_options.obj
 0002:00001884       $unwind$?dllmain_crt_dispatch@@YAHQEAUHINSTANCE__@@KQEAX@Z 0000000180005884     MSVCRT:dll_dllmain.obj
 0002:00001884       $unwind$DllMain            0000000180005884     MSVCRT:dll_dllmain_stub.obj
 0002:00001884       $unwind$__GSHandlerCheck   0000000180005884     MSVCRT:gshandler.obj
 0002:00001884       $unwind$?__scrt_uninitialize_thread_safe_statics@@YAXXZ 0000000180005884     MSVCRT:thread_safe_statics.obj
 0002:00001884       $unwind$_Init_thread_notify 0000000180005884     MSVCRT:thread_safe_statics.obj
 0002:00001884       $unwind$__scrt_acquire_startup_lock 0000000180005884     MSVCRT:utility.obj
 0002:00001884       $unwind$__scrt_dllmain_after_initialize_c 0000000180005884     MSVCRT:utility.obj
 0002:00001884       $unwind$__scrt_dllmain_before_initialize_c 0000000180005884     MSVCRT:utility.obj
 0002:00001884       $unwind$__scrt_dllmain_crt_thread_attach 0000000180005884     MSVCRT:utility.obj
 0002:00001884       $unwind$__scrt_dllmain_crt_thread_detach 0000000180005884     MSVCRT:utility.obj
 0002:00001884       $unwind$__scrt_dllmain_uninitialize_c 0000000180005884     MSVCRT:utility.obj
 0002:00001884       $unwind$__scrt_dllmain_uninitialize_critical 0000000180005884     MSVCRT:utility.obj
 0002:00001884       $unwind$atexit             0000000180005884     MSVCRT:utility.obj
 0002:0000188c       $unwind$__GSHandlerCheckCommon 000000018000588c     MSVCRT:gshandler.obj
 0002:00001898       $xdatasym                  0000000180005898     MSVCRT:amdsecgs.obj
 0002:0000189c       $unwind$?dllmain_crt_process_attach@@YAHQEAUHINSTANCE__@@QEAX@Z 000000018000589c     MSVCRT:dll_dllmain.obj
 0002:000018d8       $unwind$?fin$0@?0??dllmain_crt_process_attach@@YAHQEAUHINSTANCE__@@QEAX@Z@4HA 00000001800058d8     MSVCRT:dll_dllmain.obj
 0002:000018d8       $unwind$?fin$0@?0??dllmain_crt_process_detach@@YAH_N@Z@4HA 00000001800058d8     MSVCRT:dll_dllmain.obj
 0002:000018d8       $unwind$?fin$1@?0??dllmain_crt_process_detach@@YAH_N@Z@4HA 00000001800058d8     MSVCRT:dll_dllmain.obj
 0002:000018e0       $unwind$?dllmain_crt_process_detach@@YAH_N@Z 00000001800058e0     MSVCRT:dll_dllmain.obj
 0002:00001934       $unwind$?dllmain_dispatch@@YAHQEAUHINSTANCE__@@KQEAX@Z 0000000180005934     MSVCRT:dll_dllmain.obj
 0002:0000195c       $unwind$?filt$0@?0??dllmain_dispatch@@YAHQEAUHINSTANCE__@@KQEAX@Z@4HA 000000018000595c     MSVCRT:dll_dllmain.obj
 0002:00001964       $unwind$_DllMainCRTStartup 0000000180005964     MSVCRT:dll_dllmain.obj
 0002:00001974       $unwind$__scrt_is_nonwritable_in_current_image 0000000180005974     MSVCRT:utility.obj
 0002:00001994       $unwind$__scrt_is_nonwritable_in_current_image$filt$0 0000000180005994     MSVCRT:utility.obj
 0002:0000199c       $unwind$__scrt_dllmain_exception_filter 000000018000599c     MSVCRT:utility.obj
 0002:000019b0       $unwind$__scrt_fastfail    00000001800059b0     MSVCRT:utility_desktop.obj
 0002:000019c0       $unwind$__report_gsfailure 00000001800059c0     MSVCRT:gs_report.obj
 0002:000019c8       $unwind$capture_previous_context 00000001800059c8     MSVCRT:gs_report.obj
 0002:000019d4       $unwind$__security_init_cookie 00000001800059d4     MSVCRT:gs_support.obj
 0002:000019e0       $unwind$__isa_available_init 00000001800059e0     MSVCRT:cpu_disp.obj
 0002:000019f0       $xdatasym                  00000001800059f0     MSVCRT:guard_dispatch.obj
 0002:000019f8       $xdatasym                  00000001800059f8     MSVCRT:guard_xfg_dispatch.obj
 0002:00001a00       .edata                     0000000180005a00     getstacktr06.exp
 0002:00001a28       rgpv                       0000000180005a28     getstacktr06.exp
 0002:00001a30       rgszName                   0000000180005a30     getstacktr06.exp
 0002:00001a38       rgwOrd                     0000000180005a38     getstacktr06.exp
 0002:00001a3c       szName                     0000000180005a3c     getstacktr06.exp
 0002:00001a4d       $N00001                    0000000180005a4d     getstacktr06.exp
 0002:00001a5a       $N00002                    0000000180005a5a     getstacktr06.exp
 0002:00001ee4       .idata$6                   0000000180005ee4     kernel32:KERNEL32.dll
 0002:00001f3e       .idata$6                   0000000180005f3e     vcruntime:VCRUNTIME140.dll
 0002:0000207e       .idata$6                   000000018000607e     ucrt:api-ms-win-crt-stdio-l1-1-0.dll
 0002:0000209e       .idata$6                   000000018000609e     ucrt:api-ms-win-crt-string-l1-1-0.dll
 0002:000020c0       .idata$6                   00000001800060c0     ucrt:api-ms-win-crt-runtime-l1-1-0.dll
 0003:00000000       ?UNNAMED_STR@?1??get_thread_name@@YAPEADPEAU_jvmtiEnv@@PEAUJNIEnv_@@PEAV_jobject@@@Z@4PEBDEB 0000000180007000     libgetstacktr06.obj
 0003:00000010       expected_platform_frames   0000000180007010     libgetstacktr06.obj
 0003:000000c0       expected_virtual_frames    00000001800070c0     libgetstacktr06.obj
 0003:00000218       ?UNNAMED_LEN@?1??get_thread_name@@YAPEADPEAU_jvmtiEnv@@PEAUJNIEnv_@@PEAV_jobject@@@Z@4_KA 0000000180007218     libgetstacktr06.obj
 0003:00000220       ?$TSS0@?1??get_thread_name@@YAPEADPEAU_jvmtiEnv@@PEAUJNIEnv_@@PEAV_jobject@@@Z@4HA 0000000180007220     libgetstacktr06.obj
 0003:00000230       jvmti                      0000000180007230     libgetstacktr06.obj
 0003:00000238       mid                        0000000180007238     libgetstacktr06.obj
 0003:00000240       callbacks                  0000000180007240     libgetstacktr06.obj
 0003:00000378       ?g_tss_cv@@3U_RTL_CONDITION_VARIABLE@@A 0000000180007378     MSVCRT:thread_safe_statics.obj
 0003:00000380       ?g_tss_event@@3PEAXEA      0000000180007380     MSVCRT:thread_safe_statics.obj
 0003:00000388       ?g_tss_mutex@@3U_RTL_CRITICAL_SECTION@@A 0000000180007388     MSVCRT:thread_safe_statics.obj
 0003:000003b0       ?g_sleep_condition_variable_cs@@3P6AHPEAU_RTL_CONDITION_VARIABLE@@PEAU_RTL_CRITICAL_SECTION@@K@ZEA 00000001800073b0     MSVCRT:thread_safe_statics.obj
 0003:000003b8       ?g_wake_all_condition_variable@@3P6AXPEAU_RTL_CONDITION_VARIABLE@@@ZEA 00000001800073b8     MSVCRT:thread_safe_statics.obj
 0003:000003c4       ?__proc_attached@@3HA      00000001800073c4     MSVCRT:dll_dllmain.obj
 0003:000003d8       ?is_initialized_as_dll@@3_NA 00000001800073d8     MSVCRT:utility.obj
 0003:000003d9       ?module_local_atexit_table_initialized@@3_NA 00000001800073d9     MSVCRT:utility.obj
 0003:000003e0       ?module_local_atexit_table@@3U_onexit_table_t@@A 00000001800073e0     MSVCRT:utility.obj
 0003:000003f8       ?module_local_at_quick_exit_table@@3U_onexit_table_t@@A 00000001800073f8     MSVCRT:utility.obj
 0003:00000420       GS_ExceptionRecord         0000000180007420     MSVCRT:gs_report.obj
 0003:000004c0       GS_ContextRecord           00000001800074c0     MSVCRT:gs_report.obj
